:100000000C9424020C9468020C9468020C9468020C
:100010000C9468020C9468020C9468020C946802B8
:100020000C9468020C9468020C94090D0C94DB0D7E
:100030000C9468020C9468020C9468020C94680298
:100040000C9468020C94E5210C9468020C946802EC
:100050000C9468020C94781B0C9468020C9468024F
:100060000C9468020C9468020C9468020C94680268
:100070000C9468020C9468020C9468020C94680258
:100080000C9468020C9468020C9468020C94680248
:100090000C9468020C9468020C9468020C94680238
:1000A0000C9468020C9468020C946802480E6A0E64
:1000B000580F6A0E580FAF0ED20E580F270F3A0F77
:1000C00009120912381238126E128E12BF13BF13A2
:1000D0009912BF1349134913B013BF13BF13B913B8
:1000E00056135613561356135613561356135613C8
:1000F00056135613561356135613561356135613B8
:10010000681375137C1383138D1323024C0039007D
:10011000E100640000001E00140004001D714A008C
:1001200039001F001A0016001B734E002A00200021
:100130000800070006744B002B0021001500090081
:1001400019004D006400220017000A00050000009D
:100150006574AE0001540000007F0000E300AB00B6
:100160000154000000770000E20023001C000B0097
:10017000110000002971240018000D00100050002B
:10018000E60025000C000E00360051002800260075
:1001900012000F00370052002C002700130033001C
:1001A00038004F0031002D002F003400E5002900F9
:1001B00000000100010001000100010000003A0000
:1001C0000100F700FB00010001003B00F400F20019
:1001D000FA00FD00F5003C00F000F100F900FE001F
:1001E000F4003D00F500F300FC00FF0001003E00BC
:1001F0000100F800F600000001000100010000000D
:1002000001000000010001000100000001000000E9
:1002100001003F0001000100B400000001004000A7
:10022000AA00AC00B600010001004100A800AD002A
:10023000B5000100B7004200A900AE00B9000100FE
:10024000B60043000100AB00B7000100010044000C
:100250004500010001000100000016034500720086
:1002600067006F0044006F007800200045005A00CE
:10027000000016034500720067006F0044006F0025
:100280007800200045005A00000004030904090218
:100290006D00040100A0FA0904000001030101003F
:1002A000092111010001223F000705810308000A0E
:1002B00009040100010301020009211101000122CA
:1002C0004D000705820308000A090402000103002B
:1002D00000000921110100012236000705830308EF
:1002E000000A0904030001030000000921110100B4
:1002F00001223900070584031000011201100100DA
:10030000000008EDFE0713010001020001050109CC
:1003100006A101050719E029E715002501950875D3
:1003200001810205081901290595057501910295BC
:10033000017503910105071900297715002501951D
:100340007875018102C005010980A10185021601AD
:100350000026B7001A01002AB70075109501810028
:10036000C0050C0901A1018503160100269C021A93
:1003700001002A9C02751095018100C00501090247
:10038000A1010901A100050919012905150025018F
:1003900095057501810295017503810105010930FB
:1003A00009311581257F9502750881060938158167
:1003B000257F950175088106050C0A3802158125EF
:1003C0007F950175088106C0C005010906A10105D8
:1003D0000719E029E71500250195087501810295A7
:1003E0000175088101050819012905950575019117
:1003F000029501750391010507190029FF150025D4
:10040000FF950675088100C0000000000000000094
:10041000000000010204060A0F17202C3A4A5D7101
:10042000879DB3C7DAE9F5FCFFFCF5E9DAC7B39DB0
:1004300087715D4A3A2C20170F0A0604020100005A
:10044000000000000000000011241FBECFEFDAE022
:10045000DEBFCDBF04B603FE24C08091FB019091A6
:10046000FC01A091FD01B091FE018730904BA740A7
:10047000B04BB9F41092FB011092FC011092FD01F7
:100480001092FE0114BE84B7877F84BF88E10FB647
:10049000F89480936000109260000FBEE0E0FFE3EC
:1004A000099511E0A0E0B1E0E8E5F7E402C00590AD
:1004B0000D92A433B107D9F711E0A4E3B1E001C074
:1004C0001D92AB3FB107E1F70E944D0A0C94AA239D
:1004D0000C9400001092B9008AE08093B80008954F
:1004E00094EA9093BC009091BC0097FFFCCF909150
:1004F000B900987F983021F0903111F081E0089593
:100500008093BB0084E88093BC008091BC0087FF8F
:10051000FCCF8091B900887F883111F0803471F769
:1005200080E0089584E98093BC008091BC0084FD44
:10053000FCCF08958093BB0084E88093BC00809139
:10054000BC0087FFFCCF9091B900987F81E0983282
:1005500009F480E0089584E88093BC008091BC0099
:1005600087FFFCCF8091BB0008958091010181112C
:1005700015C080E40E9470028093010181110CC0BB
:1005800082E10E949A0280930101811105C08FEFE0
:100590000E949A02809301010E94920284B1807F9E
:1005A00084B985B1807F85B98AB1837F8AB98BB1DF
:1005B000837F8BB93E98469808950E94700480937B
:1005C00001010E94B50280B38C7080BB81B3836F40
:1005D00081BBA5E3B1E0E3E4F1E08EE08E0F119280
:1005E0001D928E13FCCF0C945A04BF92CF92DF92CF
:1005F000EF92FF920F931F93CF93DF9380910101AE
:10060000882379F0809134018F5F809334018111C8
:1006100008C00E94700480930101811102C00E94F1
:10062000020405E311E0C0E0D0E0DD24D39482E0D1
:10063000C82EEE24E394F12CC730D10500F580914B
:100640000101811164C080E40E9470028093010165
:10065000811112C082E10E949A02809301018111EE
:100660000BC0C7010C2E01C0880F0A94EAF78095D1
:100670000E949A02809301010E94920248C0CA30EF
:10068000A1F028F4C83059F0C93061F005C0CC3071
:1006900089F070F0CD3089F0209A289810C0219A06
:1006A00029980DC0229A2A980AC0239A2B9807C02D
:1006B000529A01C0539A5B9802C03E9A469890EABB
:1006C0009A95F1F79FB1799902C082E001C080E06C
:1006D00091709D25982B7C9902C084E001C080E038
:1006E000892B7D9902C038E001C030E0832B7E99D0
:1006F00002C020E101C020E0822B9FB19095991F9C
:100700009927991F9295990F907E892B0FC0809100
:100710000101811149C080E40E94700280930101AF
:10072000882379F1B12C0E9492028B2DF8019081DF
:10073000981719F08083C09200010E94B50221969B
:100740000F5F1F4FCE30D10509F076CF80910001A9
:10075000882361F1815080930001882339F08FE96B
:100760009FE00197F1F700C0000020C0A3E4B1E0D2
:10077000E5E3F1E0CF01825F91919D938E13FCCF71
:1007800015C083E10E949A02809301018111CACFB2
:1007900081E40E947002809301018111C3CF0E9405
:1007A000AB02B82EB094BFCF80E0C0CF0E9400044F
:1007B00081E0DF91CF911F910F91FF90EF90DF903B
:1007C000CF90BF900895E82FF0E0ED5BFE4F808161
:1007D000089508950F931F93CF93DF93C3E4D1E05F
:1007E00010E00C2F025F899190E00E949E1A180F72
:1007F0000C13F9CF812FDF91CF911F910F910895A5
:100800000C94D00456985E9825982D9826982E988A
:1008100027982F988FEF90E090938900809388001D
:1008200090938B0080938A0090938D0080938C002E
:10083000259A2D9A2FEF80E792E02150804090403A
:10084000E1F700C00000269A2E9A2FEF80E792E091
:10085000215080409040E1F700C00000279A2F9A75
:100860002FEF80E792E0215080409040E1F700C0F8
:10087000000025982D982FEF80E792E021508040CE
:100880009040E1F700C0000026982E982FEF80E7F7
:1008900092E0215080409040E1F700C0000027988E
:1008A0002F9856985E9825982D9826982E982798D8
:1008B0002F98089589EA8093800089E080938100D1
:1008C00024982C983F988AB18F748AB96E98479A69
:1008D0008BB1806B8BB9769A0E9402040C94CF0482
:1008E00080E2809301018091510181110EC00E942C
:1008F0006A0281E0809351012FEF83ED90E3215054
:1009000080409040E1F700C0000080E40E94700247
:100910008093010181112EC00E949A0280930101EF
:10092000811128C00E949A0280930101811122C086
:100930008FE30E949A028093010181111BC00E94E3
:10094000920280E40E94700280930101811112C022
:100950008CE00E949A028093010181110BC00E94D9
:100960009A0280930101811105C08FE30E949A02CF
:10097000809301010E94920280910101089561110A
:100980000BC0FC018281882321F085EE0E94AD100E
:1009900003C085EE0E94751180E090E008950895EF
:1009A0006091BD017091BE018091BF019091C00125
:1009B0000E94AA1A56985E9825982D9826982E98E7
:1009C00027982F98813019F4269A2E9A08955698D0
:1009D0005E98089581E0089581E008950C94EC04F8
:1009E00008950F931F93CF93DF938C01FC01C08177
:1009F000D181CE010E942319BE010E949A05EC010B
:100A0000B8010E94EE04882309F48DC0F8018281A8
:100A1000882309F44AC080915D0181111FC0C4314F
:100A2000F0E5DF0709F051C00E94F00481E08093F7
:100A30005D010E94421B90935C0180935B011092C8
:100A400054011092560110925501109258011092C3
:100A5000570110925A011092590165C080915B01B3
:100A600090915C010E944E1B883C910570F480912E
:100A70005401E82FF0E0EE0FFF1FEB5AFE4FD18339
:100A8000C0838F5F809354014EC0C43880E5D8077F
:100A900021F0C538D04501F13AC0F80182818823A0
:100AA00041F01092520182E01EC0C438E0E5DE073A
:100AB00059F580915201811106C086E20E94AD1065
:100AC00086E20E94751182E01CC0C438F0E5DF07A1
:100AD00041F3C538D045D9F4F8018281882331F03B
:100AE0001092530180E20E94C4111DC080915301F5
:100AF000811106C087E20E94AD1087E20E94751145
:100B000080E20E94CB110FC0C538D04529F381E0A7
:100B10008093520180935301C801DF91CF911F91BF
:100B20000F910C94EA0480E0DF91CF911F910F9117
:100B30000895089596E0799FF001112494E5899F26
:100B4000E00DF11D1124E60FF11DEE0FFF1FE65F12
:100B5000FE4F859194910895880F991FFC01E657E7
:100B6000F040859194910895880F991FFC01E65FEC
:100B7000FE4F8591949108950F931F93CF93DF9328
:100B8000EC01811520E3920750F5C11580E2D807EA
:100B900008F0C3C0CB3BD10590F4C83AD10508F0AA
:100BA0006AC0C53AD10508F05BC0C430D10508F071
:100BB000D0C1219709F0CAC101E010E00AC2CF3FBD
:100BC000D10511F008F0C5C1C03FD10508F0A2C0A1
:100BD000CE01805E9109089708F4BBC1B7C1C1304E
:100BE00090E5D90709F4A2C020F5C0318FE4D807F9
:100BF00070F4C11590E4D90708F094C0C11521E341
:100C0000D20708F0A3C1DD278E01106CE2C1C11527
:100C1000D04509F09BC10E942A148FEF94E32CE089
:100C2000815090402040E1F700C000000E949D1BD1
:100C3000D0C1C11597E5D90758F4C03121E5D207D5
:100C400008F01CC1C43180E5D80708F475C07EC126
:100C5000CE0190578115904108F078C1DF7073C1C3
:100C6000C53AD10509F477C1C63AD10509F076C174
:100C700002E810E4AEC1C83AD10509F472C1C93A1C
:100C8000D10509F471C1CA3AD10509F470C1CB3A52
:100C9000D10509F46FC1CC3AD10509F46EC1CD3A42
:100CA000D10509F46DC1C03BD10509F46CC1CE3A40
:100CB000D10509F46BC1CF3AD10509F46AC1C13B32
:100CC000D10509F469C1C23BD10509F468C1C33B30
:100CD000D10509F467C1C43BD10509F466C1C53B20
:100CE000D10509F465C1C63BD10509F464C1C73B10
:100CF000D10509F463C1C83BD10509F462C1C93B00
:100D0000D10509F461C1CA3BD10509F460C100E015
:100D100014E45FC18E0110655CC1CE019F700E941A
:100D2000B40558C1DF708E01106A53C18091DA0199
:100D300081608093DA014DC10E94421D811102C081
:100D40000E94281D0E945F1D90E09093FB018093FC
:100D5000FA01C23080E5D80721F48091FA01816060
:100D600086C0C43090E5D90721F48091FA018260F1
:100D70007EC0C63020E5D20721F48091FA0184605C
:100D800076C0C83080E5D80719F48091FA0127C0F1
:100D9000CA3090E5D90721F48091FA01806167C0DB
:100DA000CC3020E5D20721F48091FA0180625FC047
:100DB000CE3080E5D80721F48091FA01806457C0D5
:100DC000C03190E5D90721F48091FA0180684FC0C5
:100DD000C23120E5D20729F48091FA01846088604D
:100DE00046C0C33080E5D80721F48091FA018E7F98
:100DF0003EC0C53090E5D90721F48091FA018D7F7E
:100E000036C0C73020E5D20721F48091FA018B7FEC
:100E10002EC0C93080E5D80719F48091FA0126C0A8
:100E2000CB3090E5D90721F48091FA018F7E1FC065
:100E3000CD3020E5D20721F48091FA018F7D17C0D3
:100E4000CF3080E5D80721F48091FA018F7B0FC065
:100E5000C13190E5D90721F48091FA018F7707C05D
:100E6000C331D04531F48091FA018B7F877F809325
:100E7000FA018091FA010E94631DABC08D2F992762
:100E80008F70992781309105D9F49E012370332703
:100E900002C0880F991F2A95E2F79C688E0144E0F2
:100EA000000F111F4A95E1F700271370802B912B3B
:100EB00053E0CC0FDD1F5A95E1F7C076DD272FC038
:100EC0008230910531F4DC2FCC278E01016F106A3E
:100ED00080C08330910569F4CE018370992701E0C9
:100EE00010E002C0000F111F8A95E2F7C8019C684C
:100EF0000FC084309105B9F4CE018370992701E0C9
:100F000010E002C0000F111F8A95E2F7C8019A682D
:100F100023E0CC0FDD1F2A95E1F7C07ED7708C014E
:100F20000C2B1D2B56C08530910531F4DC2FCC27BE
:100F30008E01046F106A4DC0069709F04AC0CF7148
:100F4000DD27DC2FCC278E01106243C000E010E0CB
:100F500040C08E013EC001E810E43BC003E810E44D
:100F600038C002EE14E435C009EE14E432C00AEED3
:100F700014E42FC005EB14E42CC006EB14E429C0E4
:100F800007EB14E426C00CEC14E423C00DEC14E4CD
:100F900020C003E815E41DC00AE815E41AC002E900
:100FA00015E417C004E915E414C001E216E411C009
:100FB00003E216E40EC004E216E40BC005E216E4F8
:100FC00008C006E216E405C007E216E402C00AE221
:100FD00016E4C801DF91CF911F910F91089596E01B
:100FE000799FF001112494E5899FE00DF11D1124F2
:100FF000E60FF11DEE0FFF1FE65FFE4F8591949106
:10100000803E9105E0F4803C910558F581339105CF
:1010100009F46FC048F48932910509F463C08A323B
:10102000910509F46DC072C089339105E9F08238E9
:101030009105D1F08533910509F44DC067C0833E19
:10104000910581F138F4803E9105B9F0823E910519
:10105000D9F05CC0863E910561F1873E9105A1F112
:1010600055C00E94AC0508952091FA0120FD02C0F0
:1010700021FF4CC080EE90E049C08091FA0180FFD2
:10108000F9CF89E390E042C08091FA0182FF0EC05F
:101090008091FA0184FF03C080E090E037C083EEC6
:1010A00090E034C08091FA0182FFF2CF82EE90E0AE
:1010B0002DC08091FA0183FF0BC08091FA0184FD5D
:1010C000EBCF87EE90E022C08091FA0183FFF5CF4D
:1010D00086EE90E01BC08091FA0185FF07C089E28F
:1010E00090E014C08091FA0185FFF9CF85E390E08C
:1010F0000DC08091FA0186FF07C08AE290E006C029
:101100008091FA0186FFF9CF81E390E00E94BC054F
:10111000089508950C94890880916E010895CF93E5
:10112000DF9300D01F92CDB7DEB79C018091F10113
:10113000843019F593E099833B832A839093E900E7
:101140008FEF9091E800815095FD06C095ED9A953E
:10115000F1F700008111F5CF8091E80085FF0DC007
:1011600040E050E063E070E0CE0101960E94F90A91
:101170008091E8008E778093E8000F900F900F9099
:10118000DF91CF910895CF93DF9300D01F92CDB719
:10119000DEB72091F101243021F522E029839B83E1
:1011A0008A8383E08093E9008FEF9091E80081507B
:1011B00095FD06C095ED9A95F1F700008111F5CFE8
:1011C0008091E80085FF0DC040E050E063E070E0F2
:1011D000CE0101960E94F90A8091E8008E778093F3
:1011E000E8000F900F900F90DF91CF91089520911C
:1011F000F1012430F1F422E02093E9002FEF309147
:10120000E800215035FD06C035ED3A95F1F70000B4
:101210002111F5CF2091E80025FF0BC040E050E000
:1012200065E070E00E94F90A8091E8008E77809373
:10123000E8000895CF93DF93EC019091F101943091
:1012400009F046C080910C018823D9F080910D01EE
:101250008823B9F09093E9008FEF9091E8008150D6
:1012600095FD06C095E19A95F1F700008111F5CF43
:101270008091E80085FF2CC040E050E060E170E024
:1012800017C081E08093E9008FEF9091E8008150D2
:1012900095FD06C095ED9A95F1F700008111F5CF07
:1012A0008091E80085FF14C040E050E068E070E005
:1012B000CE010E94F90A8091E8008E778093E800C1
:1012C00080E1FE01AEE5B1E001900D928A95E1F773
:1012D000DF91CF9108958091F001811109C00E94A2
:1012E0008E0C0E94EB0C8091E20084608093E200FF
:1012F00008951092F001089508950C94D2210E944F
:10130000331B0E94D8210E94910F0C948A0842E05E
:1013100061EC81E00E94080C42E061EC82E00E94F6
:10132000080C42E061EC83E00E94080C42E161ECB1
:1013300084E00C94080C8091F301833009F455C0CB
:1013400030F4813071F0823009F48EC008958A3013
:1013500009F47AC08B3009F460C0893009F09CC070
:1013600020C08091F201813A09F096C08091E80096
:10137000877F8093E8008091F6019091F701892B97
:1013800021F460E18EE591E003C060E080E090E050
:1013900070E00E94440B8091E8008B778093E80016
:1013A00008958091F201813209F076C08091F601B2
:1013B0009091F701009719F0039709F06DC08091A3
:1013C000E800877F8093E8008091E80082FD05C0F7
:1013D0008091F1018111F8CF5FC08091F10080937D
:1013E0006E018091E8008B7753C08091F201813AC1
:1013F00009F052C08091F6019091F701892B09F014
:101400004BC08091E800877F8093E8008091E800DE
:1014100080FFFCCF80910C0136C08091F2018132B7
:10142000D9F58091F6019091F701892BA9F580916A
:10143000E800877F8093E8000E943D0C8091F401D2
:1014400080930C010C942A148091F201813221F5D1
:101450008091E800877F8093E8000E943D0C809196
:10146000F50180936F0108958091F201813AA1F412
:101470008091E800877F8093E8008091E80080FFFA
:10148000FCCF80916F018093F1008091E8008E770E
:101490008093E8000C943D0C089584B7877F84BF47
:1014A00088E10FB6F89480936000109260000FBE40
:1014B00090E080E80FB6F89480936100909361000B
:1014C0000FBE0E94E00F0E948E0C0E94EB0C8091D8
:1014D000E20084608093E20078940E94710F0E9481
:1014E000E20F82E091E00E948C0F0E94C021809167
:1014F000F101853069F40E94FA1A8091EF01882386
:10150000B1F30E94251B882391F30E94E30AEFCFD9
:101510000E94E80FECCF292F332723303105C9F083
:1015200064F42130310581F02230310509F043C0E7
:101530008DE690E02EE832E042C021323105F1F034
:101540002232310541F137C082E190E02BEF32E0E9
:1015500036C099278130910541F08230910541F0E4
:10156000892B49F5EAE8F2E005C0E2E7F2E002C0C3
:10157000EAE5F2E0849190E09F0121C06430D8F464
:10158000E62FF0E0EE0FFF1FEE5DFE4F2081318170
:1015900089E090E014C0643070F470E0FB01EE0F5D
:1015A000FF1FE65EFE4F20813181FB01EA5EFE4FA8
:1015B000808190E004C080E090E020E030E0FA011B
:1015C00031832083089580E189BD82E189BD09B41A
:1015D00000FEFDCF8091D8008F7D8093D800809150
:1015E000E00082608093E0008091E00081FDFCCF0C
:1015F0000895CF92DF92EF92FF920F931F93CF93B4
:10160000DF93EC018B016A010E945C0C811133C0F5
:10161000C114D10439F0F60180819181081B190BA6
:10162000C80FD91FE12CF12C0115110519F180917A
:10163000E80085FD16C08091E8008E778093E80071
:10164000C114D10449F0F60180819181E80EF91EA0
:10165000F182E08285E00FC00E945C0C882321F3B8
:101660000AC089918093F10001501109FFEFEF1A30
:10167000FF0ADACF80E0DF91CF911F910F91FF90A9
:10168000EF90DF90CF9008952091F8013091F9010B
:101690002617370748F06115710539F42091E800E5
:1016A0002E772093E80001C0B90140E06115710573
:1016B000A9F12091F101222309F443C0253009F456
:1016C00042C02091E80023FD40C02091E80022FDA7
:1016D00032C02091E80020FFE9CF4091F300209133
:1016E000F20030E0342BFC01CF016115710559F097
:1016F0002830310540F481918093F10061507109E7
:101700002F5F3F4FF1CF41E02830310509F040E035
:101710002091E8002E772093E800C8CF4111C9CF6F
:101720000AC08091F101882361F0853061F08091D9
:10173000E80083FD0AC08091E80082FFF2CF80E0DC
:10174000089582E0089583E0089581E0089520914E
:10175000F8013091F9012617370748F06115710536
:1017600039F42091E8002E772093E80001C0B901F8
:10177000FC0120E06115710591F18091F101882350
:1017800009F440C0853009F43FC08091E80083FD32
:101790003DC08091E80082FD2FC08091E80080FF6D
:1017A000E9CF2091F3008091F20090E0922B611537
:1017B000710559F08830910540F424912093F1008F
:1017C0003196615071090196F2CF21E0089709F036
:1017D00020E08091E8008E778093E800CBCF211144
:1017E000CCCF0AC08091F101882361F0853061F08F
:1017F0008091E80083FD0AC08091E80082FFF2CF6B
:1018000080E0089582E0089583E0089581E00895DE
:10181000982F973058F59093E900981739F0709108
:10182000EC002091ED005091F00003C0242F762FA2
:1018300050E021FF19C03091EB003E7F3093EB0068
:101840003091ED003D7F3093ED003091EB00316041
:101850003093EB007093EC002093ED005093F00078
:101860002091EE0027FF07C09F5FD3CF8F7080933A
:10187000E90081E0089580E008958091F20187FFFA
:1018800011C08091E80082FD05C08091F1018111B5
:10189000F8CF11C08091E8008B770BC08091F101E7
:1018A000882349F08091E80080FFF8CF8091E8001C
:1018B0008E778093E80008952091E4003091E50050
:1018C00095E64091EC00842F817040FF22C080910A
:1018D000E80080FD1CC08091F101882391F08530E3
:1018E00091F08091EB0085FD10C04091E400509193
:1018F000E5004217530729F39A01915011F784E04C
:10190000089582E0089583E0089581E0089580E0DD
:1019100008954091E80042FFDECF08950E94FC0C3C
:101920000E94040DE0EEF0E0808181608083E8EDAC
:10193000F0E080818F77808319BCA7EDB0E08C91B7
:101940008E7F8C9380818F7E80831092F00108952A
:101950000F931F93CF93DF930E94FC0C0E94040D02
:10196000C8EDD0E088818F778883888180688883FC
:1019700088818F7D888319BC1092F1011092ED014E
:101980001092EF011092EE0100EE10E0F80180815C
:101990008B7F808388818160888342E060E080E083
:1019A0000E94080CE1EEF0E080818E7F8083E2EE01
:1019B000F0E0808181608083808188608083F8018D
:1019C00080818E7F8083888180618883DF91CF9141
:1019D0001F910F910895E8EDF0E080818F7E808364
:1019E000E7EDF0E080818160808384E082BF81E068
:1019F0008093F0010C94A80CE8EDF0E080818E7FDC
:101A000080831092E20008951092DA001092E100B3
:101A100008951F920F920FB60F9211242F933F93A8
:101A20004F935F936F937F938F939F93AF93BF93E6
:101A3000EF93FF938091E10082FF0BC08091E20061
:101A400082FF07C08091E1008B7F8093E1000E94BC
:101A5000700F8091DA0080FF1FC08091D80080FF56
:101A60001BC08091DA008E7F8093DA008091D900CC
:101A700080FF0DC080E189BD82E189BD09B400FE0F
:101A8000FDCF81E08093F1010E946B0905C019BC74
:101A90001092F1010E9479098091E10080FF19C044
:101AA0008091E20080FF15C08091E2008E7F8093DC
:101AB000E2008091E20080618093E2008091D80092
:101AC00080628093D80019BC85E08093F1010E9468
:101AD0007D098091E10084FF30C08091E20084FFA5
:101AE0002CC080E189BD82E189BD09B400FEFDCF33
:101AF0008091D8008F7D8093D8008091E1008F7E07
:101B00008093E1008091E2008F7E8093E2008091DB
:101B1000E20081608093E2008091ED01882311F062
:101B200084E007C08091E30087FD02C081E001C02E
:101B300083E08093F1010E947F098091E10083FF9F
:101B400029C08091E20083FF25C08091E100877F5A
:101B50008093E10082E08093F1011092ED01809189
:101B6000E1008E7F8093E1008091E2008E7F809380
:101B7000E2008091E20080618093E20042E060E058
:101B800080E00E94080C8091F00088608093F00053
:101B90000E947C09FF91EF91BF91AF919F918F912E
:101BA0007F916F915F914F913F912F910F900FBE59
:101BB0000F901F9018951F920F920FB60F9211243D
:101BC0002F933F934F935F936F937F938F939F9345
:101BD000AF93BF93CF93DF93EF93FF93C091E9004F
:101BE000CF708091EC00D82FD17080FDD0E810929A
:101BF000E9008091F000877F8093F00078940E9444
:101C00001F0E1092E9008091F00088608093F00030
:101C1000CD2BCF70C093E900FF91EF91DF91CF9171
:101C2000BF91AF919F918F917F916F915F914F91F4
:101C30003F912F910F900FBE0F901F9018951F93FB
:101C4000CF93DF93CDB7DEB7AA970FB6F894DEBF78
:101C50000FBECDBFE2EFF1E088E08E0F9091F10072
:101C600091938E13FBCF0E949B098091E80083FF24
:101C70001FC18091F2019091F301492F50E04A3049
:101C8000510508F015C1FA01EA5AFF4F0C945A2386
:101C9000803881F0823809F00BC18091F6018F7095
:101CA0008093E9008091EB0085FB882780F91092F2
:101CB000E90006C08091EE019091EF0191118260E0
:101CC0009091E800977F9093E8008093F100109244
:101CD000F100C8C0282F2D7F09F0EAC0882319F031
:101CE000823061F0E5C08091F401813009F0E0C0FC
:101CF000933009F080E08093EF012BC08091F401D4
:101D0000811127C08091F6018F7009F4D1C08093B2
:101D1000E9002091EB0020FF1CC0933021F480915A
:101D2000EB00806214C09091EB0090619093EB0007
:101D300021E030E0A90102C0440F551F8A95E2F767
:101D40004093EA001092EA008091EB008860809353
:101D5000EB001092E9008091E800877F86C0811136
:101D6000A7C01091F4011F778091E3008078812B48
:101D70008093E3008091E800877F8093E8000E94D1
:101D80003D0C8091E80080FFFCCF8091E3008068EB
:101D90008093E300111102C082E001C083E08093D0
:101DA000F10186C08058823008F082C08091F40131
:101DB0009091F5018C3D53E0950779F583E08A8396
:101DC0008AE289834FB7F894DE01139620E03EE063
:101DD00051E2E32FF0E050935700E49120FF03C05D
:101DE000E295EF703F5FEF708E2F90E0EA3010F0D9
:101DF000C79601C0C0968D939D932F5F243149F7FC
:101E00004FBF8091E800877F8093E8006AE270E02E
:101E1000CE0101960E94440B14C0AE014F5F5F4F8C
:101E20006091F6010E948B0ABC01009709F440C042
:101E30009091E800977F9093E80089819A810E94B1
:101E4000A70B8091E8008B778093E80031C0803841
:101E500079F58091E800877F8093E8008091ED011B
:101E60008093F1008091E8008E778093E8000E94D3
:101E70003D0C1EC081111CC09091F4019230C0F441
:101E80008091E800877F8093E8009093ED010E94A5
:101E90003D0C8091ED01811106C08091E30087FD2A
:101EA00002C081E001C084E08093F1010E948709B3
:101EB0008091E80083FF0AC08091E800877F8093CB
:101EC000E8008091EB0080628093EB00AA960FB649
:101ED000F894DEBF0FBECDBFDF91CF911F91089563
:101EE0000895CF938091F1018823A1F0C091E9007A
:101EF000CF709091EC00892F817090FD80E8C82B05
:101F00001092E9008091E80083FD0E941F0ECF70BF
:101F1000C093E900CF910895909375018093740167
:101F20000895E0917401F0917501309721F00190CE
:101F3000F081E02D099480E00895E0917401F09122
:101F40007501309721F00280F381E02D0994089506
:101F5000E0917401F0917501309721F00480F581D2
:101F6000E02D099408952091720130917301821738
:101F7000930771F09093730180937201E091740163
:101F8000F0917501309721F00680F781E02D0994DA
:101F9000089520917001309171018217930771F0BB
:101FA0009093710180937001E0917401F09175013B
:101FB000309721F00084F185E02D0994089508956B
:101FC0000C94DF0F0E94391B0E94DD020C94FB1B56
:101FD0009F92AF92BF92CF92DF92EF92FF920F93B8
:101FE0001F93CF93DF9300D000D000D0CDB7DEB7E2
:101FF0000E94F5020DE010E0AA24A394B12C902ECB
:10200000802F0E94E303980129583E4F6901F9018E
:10201000F080F826A1F40150110988F78FEF898329
:102020008A831B820E94421B8160782F9D838C8350
:1020300049815A816B818D810E947F102FC09091C0
:10204000DA0191FF04C08E830E94E9038E8125E0AE
:1020500030E0A501022E01C0440F0A94EAF7E42EF5
:102060004F21C1F029839A828E2191E009F490E0FA
:102070009B830E94421B8160782F9D838C834981C2
:102080005A816B818D810E947F10F6018081E82644
:10209000E08204C021503109E0F6BDCF0E94E21E6B
:1020A000109176010E94910F1817B9F00E94910FBC
:1020B0008093760126960FB6F894DEBF0FBECDBF93
:1020C000DF91CF911F910F91FF90EF90DF90CF9014
:1020D000BF90AF909F900C948A0826960FB6F89404
:1020E000DEBF0FBECDBFDF91CF911F910F91FF904B
:1020F000EF90DF90CF90BF90AF909F900895CF93D7
:10210000DF93CDB7DEB72B970FB6F894DEBF0FBEC7
:10211000CDBF4F83588769877A878B87DE011196F9
:1021200086E0FD0111928A95E9F785E0FE01379678
:1021300001900D928A95E1F749815A816B817C81EA
:102140008D819E810E94C8162B960FB6F894DEBF33
:102150000FBECDBFDF91CF910895CF93882309F4AF
:10216000C2C0C82F823859F40E94910F81FDBBC0B4
:1021700089E30E94A2190E946F1A89E30CC0833878
:1021800079F40E94910F80FDAEC083E50E94A219F0
:102190000E946F1A83E50E94E419CF910C946F1A84
:1021A000843859F40E94910F82FD9DC087E40E94FB
:1021B000A2190E946F1A87E4EECF8CEF8C0F813A40
:1021C00048F48C2F0E94252181118DC08C2F0E94F4
:1021D000A219E3CF80E28C0F883048F4C77081E009
:1021E00001C0880FCA95EAF70E94281AD6CF8BE55E
:1021F0008C0F833078F4C53A29F0C63A31F083E881
:1022000090E005C081E890E002C082E890E0CF91C4
:102210000C94B30F88E58C0F833108F064C0C83A82
:1022200039F1C93A41F1CA3A49F1CB3A51F1CC3AC4
:1022300059F1CD3A61F1C03B69F1CE3A71F1CF3A33
:1022400079F1C13B81F1C23B89F1C33B91F1C43BC0
:1022500099F1C53BA1F1C63BA9F1C73BB1F1C83B20
:10226000B9F1C93BC1F1CA3BC9F180E090E038C087
:1022700082EE90E035C089EE90E032C08AEE90E0C8
:102280002FC085EB90E02CC086EB90E029C087EB57
:1022900090E026C08CEC90E023C08DEC90E020C054
:1022A00083E891E01DC08AE891E01AC082E991E0DC
:1022B00017C084E991E014C081E292E011C083E28A
:1022C00092E00EC084E292E00BC085E292E008C08A
:1022D00086E292E005C087E292E002C08AE292E0E4
:1022E000CF910C94C90FCF910895882309F44BC066
:1022F000823859F40E94910F81FF45C089E30E9402
:10230000A2190E946F1A89E30CC0833871F40E94ED
:10231000910F80FF38C083E50E94A2190E946F1AB6
:1023200083E50E94E4190C946F1A843859F40E94D2
:10233000910F82FF28C087E40E94A2190E946F1AA1
:1023400087E4EFCF9CEF980F913A58F390E2980F03
:10235000983050F4877091E001C0990F8A95EAF7A0
:10236000892F0E942E1ADFCF9BE5980F933020F41F
:1023700080E090E00C94B30F885A833120F480E021
:1023800090E00C94C90F0895882321F00E94281A28
:102390000C946F1A0895882321F00E942E1A0C9431
:1023A0006F1A08957F928F929F92AF92BF92CF92B1
:1023B000DF92EF92FF920F931F93CF93DF931F92C1
:1023C000CDB7DEB77C01C62E772EFC0105810295C4
:1023D0000F70128111110E94451A0E949B198823C7
:1023E00079F0112369F080E28C0D883048F082E0AA
:1023F0000E9484190E949B1991E0D82ED92601C011
:10240000D12CE72DE295EF70F0E0E05AFF4F0C94ED
:102410005A23872D807F072D0F70882311F0029596
:10242000007F112389F0002309F490C180E28C0D14
:10243000883020F4802F0E94281A03C0802F0E9429
:10244000381A0E946F1A82C18C2D0E9475110023C8
:1024500009F495C180E28C0D883020F4802F0E9411
:102460002E1A03C0802F0E943E1A0E946F1A87C145
:10247000972D907F872D8F70903211F08295807FFD
:10248000CC2021F0F1E0CF16B1F01EC0112349F0AD
:10249000002309F414C1013009F011C10E94581A37
:1024A0006EC1002319F0013009F469C189830E94CB
:1024B0005B1A89810AC1112321F0023008F05FC143
:1024C000FEC001115CC101C1112321F0002309F4F8
:1024D000F6C03CC1002309F4F8C03EC1872D8695A3
:1024E0008695837090E0009719F0019761F047C1DD
:1024F000112321F08C2D972D937002C080E090E085
:102500000E94B30F3CC1112321F08C2D972D9370A5
:1025100002C080E090E00E94C90F31C18C2D1123D0
:1025200019F00E94EA1D02C00E94521E0E94D71E8E
:1025300026C1872D837009F052C0111120C18C2D46
:10254000829586958770880F880F9C2D9F70892EA5
:10255000912CA12CB12C082E04C0880C991CAA1C0B
:10256000BB1C0A94D2F7C4FE14C00FE010E020E0B8
:1025700030E0B901A80104C0440F551F661F771F42
:102580008A95D2F7CB01BA016095709580959095A8
:1025900003C060E070E0CB01272D269526952370BF
:1025A00030E02230310569F02330310589F06829A7
:1025B00079298A299B292130310571F00E94101850
:1025C000DEC0682979298A299B290E942C18D7C046
:1025D0000E941018C501B4010E94F417D0C0112345
:1025E00019F0872D817001C08695882309F4C7C032
:1025F0008C2D829586958770880F880F9C2D9F70F3
:10260000892E912CA12CB12C082E04C0880C991C69
:10261000AA1CBB1C0A94D2F7C4FE14C00FE010E041
:1026200020E030E0B901A80104C0440F551F661F27
:10263000771F8A95D2F7CB01BA0160957095809586
:10264000909503C060E070E0CB01272D269526957C
:102650002370422F50E04230510569F0433051055C
:1026600089F0682979298A299B294130510571F01F
:102670000E94EA1884C0682979298A299B290E9426
:1026800006197DC00E94EA18C501B4010E94CE1847
:1026900076C08C2D90E0FC01E05EF109E531F1059A
:1026A00008F050C0E059FF4F0C945A230C2D0F70C6
:1026B000872D8F71112331F00E946718802F0E949F
:1026C000C4115DC00E948818802F0E94CB1157C092
:1026D000112339F0011153C0872D8F710E94AD185D
:1026E0004EC0023008F04BC0F7CF112339F0872DD0
:1026F0008F710E94671843C01123C9F3872D8F7112
:102700000E9488183CC0112329F0872D8F710E94E8
:10271000521835C00E94481832C0112351F0172DAD
:102720001F71812F0E94671863E0812F0E947B191F
:1027300026C081E00E948419023008F182E00E94E4
:1027400084191DC0112331F0002389F28C2D0E94C1
:10275000AD1015C0002391F28C2D0E9475110FC091
:10276000472D4F706C2DC7010E94BF040E946C174B
:1027700006C0472D4F706C2DC7010E949905DD20C2
:10278000F9F00E94771980FD1BC0F70112820E94A8
:1027900071190E946718C7010E94EF130E947119F6
:1027A0000F90DF91CF911F910F91FF90EF90DF90ED
:1027B000CF90BF90AF909F908F907F900C9488188F
:1027C0000F90DF91CF911F910F91FF90EF90DF90CD
:1027D000CF90BF90AF909F908F907F9008950F9370
:1027E0001F93CF93DF93EC01888199812B813C81EA
:1027F000232BB9F09F3F11F48F3F99F0CE010E9437
:10280000F104882371F0688179818A810E946D19B1
:102810008C010E9422190E94E917B801CE010E9482
:10282000D211DF91CF911F910F9108950E94451A07
:102830000E94551A0E941A1A0E946F1A0E94881F3D
:102840000E94D71E80E090E00E94B30F80E090E0ED
:102850000C94C90F0E94351A0C9416140E94621928
:10286000292F22952F7030E02C3031054CF42A307E
:1028700031056CF42250310922303105A8F407C02B
:102880002C30310569F02F30310551F00DC0803FFB
:1028900069F018F4803E40F409C0843F29F406C072
:1028A00093FB882780F9089580E0089581E00895DA
:1028B000CF93DF9300D000D01F92CDB7DEB70F903B
:1028C0000F900F900F900F90DF91CF910895CF93BD
:1028D000DF9300D000D000D0CDB7DEB726960FB67C
:1028E000F894DEBF0FBECDBFDF91CF9108951F9347
:1028F000CF93DF93C091850116E080918601C817C0
:1029000099F0D0E01C9FF0011D9FF00D1124E957B4
:10291000FE4F4081518162817381848195810E9443
:1029200067142196C770E9CFDF91CF911F91089569
:102930004091B7015091B8016091B9017091BA010D
:102940008091BB019091BC010C9467148091BC01F3
:1029500082958F7009F054C08091B901882309F4E1
:102960004FC080918501A09186016091B70170915F
:10297000B8014091BA015091BB01B6E08A1709F441
:102980003FC090E041155105C1F17F3F11F46F3F09
:10299000A1F1B89FF001B99FF00D1124E957FE4F46
:1029A000218172132AC02081621327C02281211144
:1029B00024C0238134812417350710F421503109B4
:1029C000241B350B283C3105C0F42091BC012F702D
:1029D00020612093BC0126E0289FF001299FF00D83
:1029E0001124E457FE4F80818F708061808387EBD4
:1029F00091E00E94EF130C94771401968770BECF7C
:102A00000895CF92DF92EF92FF920F931F93CF938F
:102A1000DF93CDB7DEB762970FB6F894DEBF0FBE77
:102A2000CDBF8C0185E0F801DE011D9601900D926D
:102A30008A95E1F7D8014C9111965C911197129605
:102A40006C9112971396CD90DC9014973091B7014A
:102A50007091B8018091BA019091BB01009709F47F
:102A60006BC17F3F19F43F3F09F466C1E090B901A3
:102A7000EE2009F4C0C02091BC01C816D90628F088
:102A8000F601E81BF90BCF0104C0809590958C0DE1
:102A90009D1DFF24F394883C910578F0F12C207F54
:102AA00009F0C6C07C2DD98AC88A89890E94581429
:102AB00087EB91E00E94EF13B1C0822F807F09F075
:102AC00046C0751314C0341312C0611110C02F70AA
:102AD00020612093BC010E94981487EB91E00E9432
:102AE000EF138091BC01D80115968C932EC0CD2890
:102AF00019F15F3F11F44F3FF9F0F62E61111CC040
:102B0000809185012091860136E0821709F45AC030
:102B100090E0389FF001399FF00D1124E957FE4FE6
:102B20007181571306C07081471303C07281711100
:102B300003C001968770E9CFF62E662309F418C109
:102B40008091BC0181608093BC01F12C11C175138F
:102B500008C0341306C0611104C08091BC01D801C3
:102B6000C3C04D875E878D859E856A8B0E942E141B
:102B70006A898823E1F16623D1F12091BC01822F7B
:102B800082958F7090E0029774F08091B7019091D8
:102B9000B80198878F831986DB86CA862C87CE0179
:102BA00007960E94EF1386E0F801A7EBB1E00190D1
:102BB0000D928A95E1F70E94A6140E949814FF24B2
:102BC000F394D6C04D875E878D859E850E946219DD
:102BD000292F22952F7030E0223031050CF0BCC037
:102BE0009F7009F0B6C0805E883008F4C1C0C8018B
:102BF0000E94EF13E4CFC816D90608F453C0F601BB
:102C0000E81BF90BCF01883C910508F450C0F12C6A
:102C10007C2DD98AC88A89890E945814E7EBF1E093
:102C200086E0DF011D928A95E9F70E949814A0C002
:102C3000751314C0341312C0611110C08091BC010F
:102C4000F8018583C8010E94EF1386E0E7EBF1E00D
:102C5000DF011D928A95E9F7FE2C8AC04D875E87B9
:102C60008D859E856A8B0E942E146A89882309F4BB
:102C7000BECF662309F4BBCF2091BC01822F829581
:102C80008F7090E002970CF48ECF8091B7019091F5
:102C9000B8019A8389831B82DD82CC822E83CE0188
:102CA00001967FCF809590958C0D9D1DACCFF62E13
:102CB000662309F49CCF75132EC034132CC02091C9
:102CC000BC0120FD1FC0822F82958F70D9F0D801E2
:102CD00015962C9315978F3049F08F5F982F92950A
:102CE000907F822F8F70892B15968C93C8010E943C
:102CF000EF1386E0F801A7EBB1E001900D928A9501
:102D0000E1F793CF86E0F801A7EBB1E001900D92D7
:102D10008A95E1F72DC04D875E878D859E850E943F
:102D20002E14811140CF8091BC0181608093BC0141
:102D3000C8010E94EF131CC0662309F458CF4D87C9
:102D40005E878D859E850E942E14882309F44FCFBF
:102D50002ACF811148CF0CC0243031050CF047CF69
:102D60009F7009F440CFF8019581907F09F03BCF27
:102D70008F2D62960FB6F894DEBF0FBECDBFDF91E8
:102D8000CF911F910F91FF90EF90DF90CF9008951A
:102D90001F93CF93DF93CDB7DEB72C970FB6F89480
:102DA000DEBF0FBECDBF4F83588769877A878B8779
:102DB0009C87CE0107960E940115882369F08F81B8
:102DC00098852A853B85232BF1F19F3F09F063C04D
:102DD0008F3F09F060C037C086E0FE013796DE0104
:102DE000119601900D928A95E1F76F817885EA85B9
:102DF000FB85309741F17F3F11F46F3F21F1209126
:102E0000860130E0C90101968770992740918501BC
:102E100050E08417950709F447C069837A83FD83DE
:102E2000EC8396E0929FD001939FB00D1124A95797
:102E3000BE4FFE01319601900D929A95E1F7809375
:102E400086010E94771416E0809185019091860199
:102E50008917C1F1189FC001112489579E4F0E9404
:102E60000115882379F1E09185011E9FF00111245D
:102E7000E957FE4F40815181628173818481958140
:102E80000E9467148091850190E0019687709927D0
:102E900080938501D9CF4F81588569857A858B8547
:102EA0009C850E946714CFCF0E942A14109286013D
:102EB00010928501E7EBF1E086E0DF011D928A9533
:102EC000E9F7C1CF2C960FB6F894DEBF0FBECDBF89
:102ED000DF91CF911F910895EF92FF920F931F936F
:102EE000CF93DF938C01009709F46CC0F12CEE2492
:102EF000E394E8012196F8018491843740F484300A
:102F000008F051C0813081F0823019F15BC0853703
:102F100009F444C0A8F19CE7980F903708F052C01C
:102F20008F770E94751141C00E5F1F4FFE01C49143
:102F300080E28C0F883048F4C7708E2D01C0880F56
:102F4000CA95EAF70E94481A14C08C2F0E94AD104F
:102F50002DC00E5F1F4FFE01C49180E28C0F8830A0
:102F600058F4C7708E2D01C0880FCA95EAF70E94E9
:102F70004E1A0E946F1A1AC08C2F0E94751116C02B
:102F80000E5F1F4FFE01C491CC2381F08FE99FE0BB
:102F90000197F1F700C00000C150F6CF0E5F1F4F40
:102FA000FE01F49003C00E94AD108E018F2D882386
:102FB00009F49FCFEFE9FFE03197F1F700C000007F
:102FC0008150F5CFDF91CF911F910F91FF90EF903E
:102FD000089508956093C1017093C2018093C30165
:102FE0009093C4010C9416140F931F930091C10188
:102FF0001091C2012091C3013091C401DC01CB01C9
:10300000802B912BA22BB32B8093C1019093C201F3
:10301000A093C301B093C4011F910F910C94161497
:103020000F931F930091C1011091C2012091C30120
:103030003091C401DC01CB0180239123A223B3236F
:103040008093C1019093C201A093C301B093C401C6
:103050001F910F910C9416140F931F930091C101AF
:103060001091C2012091C3013091C401DC01CB0158
:1030700080279127A227B3278093C1019093C20193
:10308000A093C301B093C4011F910F910C94161427
:103090001092BD011092BE011092BF011092C001AA
:1030A0000C94161441E050E060E070E004C0440F5E
:1030B000551F661F771F8A95D2F74093BD01509325
:1030C000BE016093BF017093C0010C94161441E0DF
:1030D00050E060E070E004C0440F551F661F771F8A
:1030E0008A95D2F78091BD019091BE01A091BF0158
:1030F000B091C001482B592B6A2B7B2B4093BD010B
:103100005093BE016093BF017093C0010C941614DC
:1031100041E050E060E070E004C0440F551F661FBE
:10312000771F8A95D2F7409550956095709580915C
:10313000BD019091BE01A091BF01B091C001482393
:1031400059236A237B234093BD015093BE016093B2
:10315000BF017093C0010C94161441E050E060E090
:1031600070E004C0440F551F661F771F8A95D2F781
:103170008091BD019091BE01A091BF01B091C001AD
:10318000482759276A277B274093BD015093BE01EA
:103190006093BF017093C0010C9416140F931F939A
:1031A0000091BD011091BE012091BF013091C0017D
:1031B000DC01CB01802B912BA22BB32B8093BD0183
:1031C0009093BE01A093BF01B093C0011F910F91D6
:1031D0000C9416140F931F930091BD011091BE0122
:1031E0002091BF013091C001DC01CB0180239123EC
:1031F000A223B3238093BD019093BE01A093BF018E
:10320000B093C0011F910F910C9416140F931F934C
:103210000091BD011091BE012091BF013091C0010C
:10322000DC01CB0180279127A227B3278093BD0122
:103230009093BE01A093BF01B093C0011F910F9165
:103240000C9416140895CF92DF92EF92FF920F9391
:103250001F93CF93DF938C01C090C101D090C20126
:10326000E090C301F090C4018091BD019091BE0136
:10327000A091BF01B091C001C82AD92AEA2AFB2A2D
:10328000CFE1D0E0D701C6010C2E04C0B695A795BA
:10329000979587950A94D2F780FF06C0B8018C2FC6
:1032A0000E94EF07019721F4219760F780E001C0A9
:1032B0008C2FDF91CF911F910F91FF90EF90DF90B6
:1032C000CF900895CF93DF93EC010E942319BE01A4
:1032D0000E94EF07DF91CF910895CB010E94621900
:1032E00008958091C501859585958595089580916E
:1032F000C5018770089598E0899F90011124262BBD
:103300002093C5010C9467182091C50180958223F4
:103310008093C501982F977069F430E0482F5527A6
:1033200047FD50952417350729F085958595859596
:103330000C94881808959091C501977081E009F464
:1033400080E0089590910C01992321F090910D0156
:10335000911109C020910E0130910F01F9013296AF
:103360009FEF40E01FC0982F9695969596959F30B9
:1033700050F5E0910E01F0910F01E90FF11D8770FA
:1033800021E030E0A90102C0440F551F8A95E2F701
:10339000CA019181892B818308959F3F39F04F5F46
:1033A0004E3041F051915813F8CF0DC05111F7CF65
:1033B000942FF5CF9F3F39F0F901E90FF11D97FDEB
:1033C000FA9582830895089590910C01992321F034
:1033D00090910D01911109C020910E0130910F01C2
:1033E000F9013296205F3F4F1FC0982F9695969512
:1033F00096959F30F0F4E0910E01F0910F01E90FE6
:10340000F11D877021E030E0A90102C0440F551F73
:103410008A95E2F7CA018095918189238183089575
:103420003196E217F30729F090819813F9CF1082B3
:10343000F7CF089581E090E0E0910E01F0910F0147
:10344000E80FF91F1082019680319105A9F70895C0
:103450009091D901892B8093D901089580959091FD
:10346000D90189238093D90108951092D901089533
:103470009091D801892B8093D801089580959091DF
:10348000D80189238093D80108951092D801089516
:103490009091D701892B8093D701089580959091C1
:1034A000D70189238093D70108951092D7010895F9
:1034B0008093C60108951092C601089580910E016F
:1034C00090910F01FC0131969C01205F3F4F80E0FD
:1034D000919191118F5FE217F307D1F70895E09171
:1034E0000E01F0910F018091D9018083E0910E01CE
:1034F000F0910F0190818091D801892B8083E09118
:103500000E01F0910F0190818091D701892B80836A
:103510008091C601882361F0E0910E01F0910F01C6
:103520009081892B80830E945E1A81111092C601BE
:1035300080910E0190910F010C949D0F20E0009757
:1035400039F0AC0141505109842395232F5FF7CF07
:10355000822F0895CF92DF92EF92FF926C01EE24BA
:10356000FF24C114D104E104F10421F0C701B60124
:1035700020E101C020E0C72ED82EE92EFF24C1147F
:10358000D104E104F10419F0285FC701B6016B0111
:103590007C0154E0F694E794D794C7945A95D1F7F8
:1035A000C114D104E104F10419F02C5FC701B60184
:1035B0006B017C0142E0F694E794D794C7944A9556
:1035C000D1F7C114D104E104F10419F02E5FC70151
:1035D000B601DC01CB01B695A79597958795892B08
:1035E0008A2B8B2B09F02F5F822FFF90EF90DF90BB
:1035F000CF9008958091F101843021F11092DB0188
:1036000020E488E190E00FB6F894A89580936000DC
:103610000FBE2093600080E00E948A0883B7817FFC
:10362000846083BF83B7816083BF7894889583B7B4
:103630008E7F83BF88E10FB6F8948093600010926C
:1036400060000FBE0895089508950E94231B0E94F4
:10365000F5020E94241B0E94EA0391E0811101C03F
:1036600090E0892F08950E942A140E94910F0C94D3
:103670008A0882E084BD93E095BD9AEF97BD809360
:103680006E0008952FB7F8948091DC019091DD01D0
:10369000A091DE01B091DF012FBF0895CF92DF929C
:1036A000EF92FF920F931F932FB7F8944091DC0194
:1036B0005091DD016091DE017091DF012FBF6A0141
:1036C0007B01EE24FF248C0120E030E0C016D106FF
:1036D000E206F30610F4415051099A01281B390BF8
:1036E000C9011F910F91FF90EF90DF90CF90089547
:1036F0001F920F920FB60F9211248F939F93AF9347
:10370000BF938091DC019091DD01A091DE01B09129
:10371000DF010196A11DB11D8093DC019093DD01B5
:10372000A093DE01B093DF01BF91AF919F918F9184
:103730000F900FBE0F901F9018950E948E0CF8945A
:103740002FEF87EA91E6215080409040E1F700C0DA
:10375000000087E090EBDC018093FB019093FC017B
:10376000A093FD01B093FE019CE088E10FB6F894B0
:10377000A895809360000FBE90936000FFCFEF92FA
:10378000FF920F931F93CF93DF93D82FCDE08C2F11
:103790000E94E30305E010E0E82EF12CC701002EA3
:1037A00002C0959587950A94E2F780FF09C0602FC3
:1037B0007C2F80E00E949A05D81302C081E006C0E9
:1037C0000150110958F7C15010F780E0DF91CF91F7
:1037D0001F910F91FF90EF900895CF93C82F8CE227
:1037E0000E94BF1B882321F08C2FCF910C94BF1B0C
:1037F00080E0CF910895CF930E94421D811102C0B5
:103800000E94281DC5E6C15049F00E94F5028FE3D1
:103810009CE90197F1F700C00000F5CF89E20E9412
:10382000ED1B811113C18AE20E94ED1B81110E94E0
:10383000281D85E00E94ED1B81110E949D1B0E94A6
:103840004D1D8093DA0187E00E94ED1B8823A9F1CA
:103850008BE10E94ED1B882351F08091DA0181FBFE
:10386000222720F991E0922790FB81F90EC08EE08B
:103870000E94ED1B882361F08091DA0182FB2227F0
:1038800020F991E0922790FB82F98093DA0115C02C
:1038900080E10E94ED1B9091DA01882341F093FBB7
:1038A000222720F981E0822780FB93F904C0892F29
:1038B000809580FB90F99093DA018091DA010E9463
:1038C000511D0E945F1D8093FA0180EE0E94ED1B46
:1038D000882341F08091FA01982F909590FB80F910
:1038E0008093FA0189E30E94ED1B882359F08091AF
:1038F000FA0181FB222720F991E0922790FB81F9C0
:103900008093FA0182EE0E94ED1B882359F080918A
:10391000FA0182FB222720F991E0922790FB82F99D
:103920008093FA0186EE0E94ED1B882359F0809166
:10393000FA0183FB222720F991E0922790FB83F97B
:103940008093FA0183EE0E94ED1B882359F0809149
:10395000FA0184FB222720F991E0922790FB84F959
:103960008093FA0185E30E94ED1B882359F0809132
:10397000FA0185FB222720F991E0922790FB85F937
:103980008093FA0181E30E94ED1B882359F0809116
:10399000FA0186FB222720F991E0922790FB86F915
:1039A0008093FA0181E10E94ED1B882359F08091F8
:1039B000FA0187FB222720F991E0922790FB87F9F3
:1039C0008093FA018091FA010E94631D8091FA01AF
:1039D00087FB882780F980930D0187E20E94ED1B09
:1039E000C82F8EE10E94ED1B8111C2608FE10E9401
:1039F000ED1B8111C46080E20E94ED1B8111C86043
:103A000081E20E94ED1B8111C06182E20E94ED1BE8
:103A10008111C06283E20E94ED1B8111C06484E2C7
:103A20000E94ED1B882311F0C06802C0CC2329F04E
:103A30008C2F0E945A1D6C2F03C00E94561D682FA8
:103A400070E080E090E0CF910C94EA17CF91089558
:103A50006DEE7EEF80E090E00E94942360E082E0D3
:103A600090E00E94822360E083E090E00E94822345
:103A700060E084E090E00E94822360E085E090E0D6
:103A80000C94822380E090E00E947C2321E08D3E14
:103A90009E4F09F020E0822F089582E090E00C9480
:103AA0007423682F82E090E00C94822383E090E0FE
:103AB0000C947423682F83E090E00C94822384E0BC
:103AC00090E00C947423682F84E090E00C9482239F
:103AD0008091E20180FF0BC06091130185E0689F37
:103AE000B001112475956795759567952BC081FF79
:103AF00009C06091130185E0689FB001112475959C
:103B0000679520C082FF07C06091130185E0689F20
:103B1000B001112417C09091E3019923D1F0609175
:103B20001201961788F72091130185E0289F9001D4
:103B30001124929FA001939F500D112470E0CA019F
:103B40000E9446236038710540F46115710539F013
:103B500002C065E070E0862F08958FE7089581E048
:103B600008958091E20180FF08C06091110170E02A
:103B7000759567957595679521C081FF06C0609121
:103B8000110170E07595679519C082FF04C06091BE
:103B9000110170E010C09091E3019923C1F0609190
:103BA00010019617A0F780911101899FC00111247F
:103BB00070E00E9446236038710528F46115710594
:103BC00021F0862F08958FE7089581E0089561E040
:103BD00070E0F4CF803F21F40E94681D819504C0FD
:103BE000813F29F40E94681D8093E6010895823F79
:103BF00021F40E94681D819504C0833F29F40E942E
:103C0000681D8093E5010895893F19F40E94B11D54
:103C100005C08A3F31F40E94B11D81958093E70170
:103C200008958B3F21F40E94B11D819504C08C3F03
:103C300029F40E94B11D8093E8010895843F21F486
:103C40008091E401816017C0853F21F48091E401F7
:103C5000826011C0863F21F48091E40184600BC032
:103C6000873F21F48091E401886005C0883F31F4EA
:103C70008091E40180618093E40108958D3F21F4F7
:103C80008091E20181600BC08E3F21F48091E201BE
:103C9000826005C08F3F29F48091E20184608093A7
:103CA000E2010895803F39F48091E60187FF6CC0FE
:103CB0001092E60169C0813F29F48091E60118164F
:103CC000BCF362C09091E501823F29F497FF5CC08C
:103CD0001092E50159C0833F19F41916CCF354C072
:103CE000893F41F48091E70118160CF04DC0109205
:103CF000E7014AC08A3F29F48091E70187FF44C069
:103D0000F6CF8B3F39F48091E80187FF3DC01092D8
:103D1000E8013AC08C3F29F48091E8011816BCF301
:103D200033C0843F21F48091E4018E7F17C0853F2A
:103D300021F48091E4018D7F11C0863F21F48091B0
:103D4000E4018B7F0BC0873F21F48091E401877FE2
:103D500005C0883F31F48091E4018F7E8093E401B7
:103D600013C08D3F21F48091E2018E7F0BC08E3F06
:103D700021F48091E2018D7F05C08F3F29F480916D
:103D8000E2018B7F8093E2018091E50181110EC0F9
:103D90008091E60181110AC08091E701811106C07E
:103DA0008091E801811102C01092E301089584EE30
:103DB00091E00E94A80F0E94421B9093E101809322
:103DC000E00108951F93CF93DF938091E0019091DC
:103DD000E1010E944E1BAC019091E301992321F077
:103DE0002091140130E006C0209115018AE0289F3F
:103DF000900111244217530708F486C08091E50111
:103E0000C091E601D091E7011091E801811107C04E
:103E1000C11176C0D11174C0111172C075C09F3F1D
:103E200019F09F5F9093E301181624F40E94681D17
:103E30008093E5018091E50187FF05C00E94681D20
:103E400081958093E5011C1624F40E94681D8093DF
:103E5000E6018091E60187FF05C00E94681D8195FB
:103E60008093E6016091E501662339F1C091E60196
:103E7000CC2319F1772767FD7095872F972F0E9424
:103E8000572223E333E343E35FE30E94BB220E9414
:103E900024226093E5016C2F772767FD7095872FAB
:103EA000972F0E94572223E333E343E35FE30E940B
:103EB000BB220E9424226093E6011D1624F40E9476
:103EC000B11D8093E7018091E70187FF05C00E9443
:103ED000B11D81958093E701111624F40E94B11D54
:103EE0008093E8018091E80187FF05C00E94B11D21
:103EF00081958093E801DF91CF911F910C94D71E9B
:103F00009F3F09F08ECF96CFDF91CF911F910895FB
:103F1000E4EEF1E085E0DF011D928A95E9F7109269
:103F2000E3011092E2010895833081F128F4813099
:103F300059F08230D1F00895853009F449C0B8F1C4
:103F4000863009F456C0089580911501262F30E07F
:103F5000280F311D2F3F310524F4680F60931501A0
:103F600008958FEF80931501089580911401262FF5
:103F700030E0280F311D2F3F310524F4680F609386
:103F8000140108958FEF8093140108958091130117
:103F9000262F30E0280F311D2F3F310524F4680F04
:103FA0006093130108958FEF80931301089580911A
:103FB0001201262F30E0280F311D2F3F310524F448
:103FC000680F6093120108958FEF80931201089596
:103FD00080911101262F30E0280F311D2F3F310530
:103FE00024F4680F6093110108958FEF80931101FD
:103FF000089580911001262F30E0280F311D2F3FAA
:10400000310524F4680F6093100108958FEF8093B9
:1040100010010895833011F128F4813049F0823085
:1040200091F00895853081F120F18630C1F1089535
:1040300080911501681720F4861B8093150108955F
:1040400010921501089580911401681720F4861BC1
:104050008093140108951092140108958091130122
:10406000681720F4861B80931301089510921301A2
:10407000089580911201681720F4861B8093120125
:10408000089510921201089580911101681720F48B
:10409000861B80931101089510921101089580915B
:1040A0001001681720F4861B809310010895109268
:1040B000100108950F931F938D3109F46BC008F020
:1040C0003FC08E3009F47FC0C0F4873009F469C066
:1040D00068F4863009F0B1C08091DA01817F8E7F6B
:1040E0008093DA0181E08093EA01A8C0883009F466
:1040F000A2C08B3009F49FC0A0C0863109F49BC0D8
:1041000078F4803109F472C0813109F096C00E94C0
:104110002A1490910D0181E0892780930D018BC0B5
:10412000893109F488C08B3109F087C08091DA01A8
:1041300081FB222720F991E0922790FB81F94CC066
:10414000853309F470C048F4873209F46CC008F470
:1041500059C0893209F467C070C0833438F48A3397
:1041600008F04EC0883309F466C067C0833409F490
:104170005AC0883409F061C00E942A140FEF13ED71
:1041800020E3015010402040E1F700C000000E94F1
:104190009D1B51C00E94DE210E94910F0E948A083F
:1041A0004AC09091DA01892F8095817080FB90F947
:1041B00029F0966098609093DA0140C0997F977FCC
:1041C0009093DA0138C08091DA0182FB222720F92E
:1041D00091E0922790FB82F98093DA01992359F1BB
:1041E0008091DA0181608093DA0125C08091DA0143
:1041F00083FB222720F991E0922790FB83F9ECCFF3
:10420000895301C08D5141E050E060E070E08A01C7
:104210009B0104C0000F111F221F331F8A95D2F784
:10422000C901B80104C061E070E080E090E00E9444
:10423000EA170E942A1481E001C080E01F910F91CB
:10424000089580E0089580E00895CF93C82F80916D
:10425000EA01813079F018F08230E9F187C0E0910D
:104260000E01F0910F018081813169F0823209F0F5
:104270007FC009C0E0910E01F0910F018081813172
:1042800011F0823261F48C2F0E942121811104C02F
:104290008C2F0E945A201DC081E090E01AC08C2F04
:1042A0000E942321811114C0C43179F048F4CB302D
:1042B00079F0C03109F060C082E08093EA0108C063
:1042C000C93219F0C83321F057C01092EA0154C026
:1042D00081E0817053C0C93289F118F5C43171F1A0
:1042E000A8F4C73009F046C08AE08093150194E134
:1042F0009093140193E0909313018093120188E04E
:104300008093110188E28093100134C0CE51C630F1
:1043100088F5EC2FF0E0E65DFE4F80818093E901A7
:1043200029C0CE34E9F020F4CB3421F56AE013C083
:10433000C13579F0C235F1F461E00DC08091E90139
:10434000882319F01092E90115C081E08093EA01F9
:1043500015C061E006C08091E9010E94941F0AC067
:104360006AE08091E9010E940A2004C01092EA01EB
:1043700080E004C081E002C080E0ABCFCF9108951F
:10438000E1E8F0E0808188608083808181608083C3
:104390008FB7F89493E09093890090ED9093880004
:1043A0008FBF0895EFE6F0E08081826080830895FA
:1043B000EFE6F0E080818D7F80830895EFE6F0E006
:1043C000908182E08927808308951F920F920FB613
:1043D0000F9211242F933F934F935F936F937F938B
:1043E0008F939F93AF93BF93EF93FF938091EB01D4
:1043F0009091EC0101969093EC018093EB01811177
:1044000003C082E00E948A08E091EC01E695E695FF
:10441000F0E0E85FFB4FE4918091EB018E1303C065
:1044200080E00E948A08FF91EF91BF91AF919F9128
:104430008F917F916F915F914F913F912F910F904D
:104440000FBE0F901F90189504D06894B1118DC0C5
:10445000089570D088F09F5790F0B92F9927B751E1
:10446000A0F0D1F0660F771F881F991F1AF0BA9538
:10447000C9F712C0B13081F077D0B1E0089574C0AF
:10448000672F782F8827B85F39F0B93FCCF386952E
:1044900077956795B395D9F73EF49095809570958B
:1044A00061957F4F8F4F9F4F0895E89409C097FB08
:1044B0003EF490958095709561957F4F8F4F9F4FFB
:1044C0009923A9F0F92F96E9BB279395F69587953F
:1044D00077956795B795F111F8CFFAF4BB0F11F402
:1044E00060FF1BC06F5F7F4F8F4F9F4F16C08823A9
:1044F00011F096E911C0772321F09EE8872F762FDF
:1045000005C0662371F096E8862F70E060E02AF01F
:104510009A95660F771F881FDAF7880F969587950B
:1045200097F9089557FD9058440F551F59F05F3F74
:1045300071F04795880F97FB991F61F09F3F79F0C5
:1045400087950895121613061406551FF2CF469547
:10455000F1DF08C0161617061806991FF1CF8695C9
:104560007105610508940895E894BB2766277727AD
:10457000CB0197F908950BD078C069D028F06ED0A0
:1045800018F0952309F05AC05FC01124EECFCADF9E
:10459000A0F3959FD1F3950F50E0551F629FF00156
:1045A000729FBB27F00DB11D639FAA27F00DB11DAF
:1045B000AA1F649F6627B00DA11D661F829F222738
:1045C000B00DA11D621F739FB00DA11D621F839FBF
:1045D000A00D611D221F749F3327A00D611D231F95
:1045E000849F600D211D822F762F6A2F11249F57E3
:1045F00050408AF0E1F088234AF0EE0FFF1FBB1F06
:10460000661F771F881F91505040A9F79E3F5105A4
:1046100070F014C0AACF5F3FECF3983EDCF38695B0
:1046200077956795B795F795E7959F5FC1F7FE2B4F
:10463000880F911D9695879597F9089597F99F672B
:1046400080E870E060E008959FEF80EC089500241A
:104650000A941616170618060906089500240A94E7
:1046600012161306140605060895092E0394000C6D
:1046700011F4882352F0BB0F40F4BF2B11F460FFFC
:1046800004C06F5F7F4F8F4F9F4F089597FB072E9A
:1046900016F4009407D077FD09D00E94602307FC30
:1046A00005D03EF4909581959F4F08957095619542
:1046B0007F4F0895EE0FFF1F0590F491E02D0994B0
:1046C000AA1BBB1B51E107C0AA1FBB1FA617B70738
:1046D00010F0A61BB70B881F991F5A95A9F7809554
:1046E0009095BC01CD010895F999FECF92BD81BD91
:1046F000F89A992780B50895A8E1B0E042E050E02B
:104700000C949C23262FF999FECF92BD81BDF89A77
:10471000019700B4021639F01FBA20BD0FB6F89405
:10472000FA9AF99A0FBE08950196272F0E948323C3
:104730000C948223DC01CB01FC01F999FECF06C069
:10474000F2BDE1BDF89A319600B40D92415050404F
:08475000B8F70895F894FFCFBB
:1047580002208C081A09F708C3088F080101C7014D
:1047680028080A03140A3F4D3639C9037C03460357
:104778000D03A002B902D202EB02010203040506EE
:044788000708090015
:00000001FF
